:10000000073099006230B1006830B7000D30BA0097
:100010004330BF0073239223851DC62BAA0B0E28E5
:10002000AB0B0E28033034210E217B30CF004C3037
:10003000CE00CC30CD00CD30CC004F228730CF0069
:100040004830CE00CD01CC01B422FC214708D800B5
:100050004608D9004508DA002030BB00C71F332806
:100060005E232D30BB0026210330D5003E303523E2
:100070001E217C30CF003830CE005130CD00EC3026
:10008000CC004F228430CF00CE01CD01CC01B6226E
:10009000FC21A301C71F4E285E232314282103300F
:1000A000D500303035232D302318AE0005303421F3
:1000B0001E217530CF000330CE001230CD006F30DE
:1000C000CC004F228130CF000830CE00CD01CC01D2
:1000D000B4224808DB004708A3004608A4004508EE
:1000E000A5001E216E30CF000630CE003730CD0087
:1000F000BD30CC004F227A30CF001D30CE00B23060
:10010000CD002D30CC00B6224808D7004708D800D3
:100110004608D9004508DA000E216C30CF003B308C
:10012000CE00E730CD00A230CC004F221521570879
:10013000C8005808C7005908C6005A08C500B422AC
:1001400015210E214F225B08CF002308CE00240882
:10015000CD002508CC00B622FC21C71FB328C6015C
:100160000130C500BA2864304502031CBA28C60114
:100170006330C50026210230D500393035232030C8
:10018000A000A201A1019F149F18C4281E08A10766
:1001900083161E0883120310A2070318A10AAA0BD4
:1001A000CF28AB0BCF28A00BC3280E217B30CF006C
:1001B000C530CE003730CD004230CC004F228C30DD
:1001C000CF003730CE00DA30CD00AB30CC00B622D5
:1001D0000F30AF23CF001030AF23CE001130AF234C
:1001E000CD001230AF23CC00B622FC2126210530F1
:1001F000D5003630352394234130A3002308AF23A4
:100200000038031906298423A30AFE282E3084000F
:1002100000088423840A041F08290C28C701210828
:10022000C6002208C500882108004808CF004708FA
:10023000CE004608CD004508CC0008005808C7008D
:100240005908C6005A08C500882108004608C7009A
:100250004508C6000800F830D60000000000000085
:100260000000D60B30290800AC008316051183125C
:100270000515A2010516A1010511000005120000D7
:100280000516000005150830A3000512AC1F4A2909
:1002900005154B2905110516AC0DA30B45290512B3
:1002A00083160515831205160000051D58293134E3
:1002B0000512FF30A300051D61292B21A30B5B292B
:1002C00032346C212C08A1007D216C212C08A20065
:1002D0007D216C217D210800AC010830A3000516AA
:1002E0000000051D75292C1476292C100512A30B6E
:1002F0007A297C29AC0D6F29080083160511831219
:100300000511051600000512831605158312080055
:100310009630C800C901C71F90295E236423C917FE
:10032000D3014708031DA5294608C7004508C60094
:10033000C501D3154708031DA5294608C700C601F6
:10034000D311531647080319B6295308C802031DD1
:10035000031CA92A0310C71BB329C50DC60DC70D61
:10036000C80BAB29A92AC91FC7130034C701C6018E
:10037000C501C401C8010034D3014708031DDC29AD
:100380004608C7004508C6004408C500C401D31587
:100390004708031DDC294608C7004508C600C501FB
:1003A000D31153164708031DDC294608C700C601B0
:1003B000D31547080319B6295308C802031D031CA7
:1003C000A92A0310C71BEB29C40DC50DC60DC70D07
:1003D000C80BE229A92A4A1B451CB329C41FB3290B
:1003E000C50A0319C60A0319C70A031DB3296A23DC
:1003F000C80A03199E2AB32948080319003447087C
:10040000C900C7179630C802C81F432AC809C80ABE
:1004100008304802031C272AC800C50D4608C5003D
:100420004708C600C70108304802031C272AC80035
:10043000C50D4608C500C60108304802031C272A1E
:10044000C800C50DC5014808031D03102E2A480821
:1004500003192E2A03106A23C80B2A2A4A1B451C9B
:100460003A2A031C3A2AC50A0319C60A0319C70AFD
:10047000C71B432AC91F00345E2364230034C7010D
:10048000C601C50100344A14CA1FFF34C701C91F81
:10049000FF30C700C600C500C90DC70CFF344808AF
:1004A000031D4F080319B62947084E06C9004F0817
:1004B000C8077E30031C602AC80203189E2A632ADC
:1004C000C802031CA92A4708C4004608C3004508FF
:1004D000C200C417CE170310C701C601C5011830EA
:1004E000D300421C7D2A4C08C5074D0803184D0F48
:1004F000C6074E0803184E0FC7076A23C40CC30C67
:10050000C20C0310D30B712AC71B8B2AC40DC50D57
:10051000C60DC70DC8034A1B451C9B2AC41F9B2A36
:10052000C50A0319C60A0319C70A031D9B2A6A23B1
:10053000C80A03199E2AC91FC7130034CA14CA1F48
:10054000FF34FF30C800C700C600C500C90DC70C86
:10055000FF344A15CA1FFF340130C800C701C60165
:10056000C501C90DC70CFF348030CE0647084E06C2
:10057000D300C401CB0148084F02031CD72A4F08FF
:10058000C2004808CF004208C8004E08C200470811
:10059000CE004208C7004D08C2004608CD00420800
:1005A000C6004C08C2004508CC004208C5004F08F0
:1005B000031900344708C900C717CE174F0848026F
:1005C000CF0003190A2B08304F02031C002BCF0069
:1005D0004C08CB004D08CC004E08CD00CE010830B1
:1005E0004F02031C002BCF004C08CB004D08CC0061
:1005F000CD0108304F02031C002B4908C70000340E
:100600004F0803190A2B0310CE0CCD0CCC0CCB0CCD
:10061000CF0B032BD31F172BCB09CC09CD09CE0948
:10062000CB0A0319CC0A0319CD0A0319CE0A4B08C9
:10063000C4074C0803184C0FC5074D0803184D0F8D
:10064000C6074E0803184E0FC707D31B2E2B031CDB
:10065000EB296A23C40CC80FEB299E2A0318BC2976
:100660005D2362238030C90690298400CE010A30C0
:10067000CD00422342088000303080078403D50B30
:10068000362B0800C301C2011030D400470DC20D43
:10069000C30D4D08C2024E08031C4E0FC3020318BF
:1006A000582B4D08C2074E0803184E0FC3070310FE
:1006B000C60DC70DD40B462B0034C409C509C609A5
:1006C000C7090800C40A0319C50A0319C60A031991
:1006D000C70A0800C70CC60CC50C0800DD000000E6
:1006E000DD0B702B08008316FF2390008512051286
:1006F000A730810051309F0083128512C1309F00C6
:100700004030AF23DC000800DF000A30DE000310B9
:100710008512031C85165C086E230314DF0CDE0BA8
:10072000882B08000A3084230D30842B5F10851D30
:1007300000340930DE000A306E230310851D0314D7
:10074000DF0C5C086E230000DE0B9D2B5F08851913
:10075000A72B5F14080096235F1CAB2B08007F3982
:1007600083169B001C141A08831208003F39831655
:100770009B008B131C1555309D00AA309D009C14C6
:100780001C118B179C18C22B8312080092233E3039
:10079000842396235F1CA3001B3A0319D02BC92B7B
:1007A000AB23A300443A0319DE2B2308553A03195F
:1007B000E92B23084D3A03190E28C92BA301AB23BB
:1007C00083169A0083122308B623A30A231FDF2B64
:1007D000C62B40308423A3012308AF238423A30A1C
:0607E000231FEC2BC62BC9
:02400E0084111B
:104200005000720065007300730075007200650055
:104210002D0046004C004F00330032003A0086006B
:104220003E0000000000480075006D006900640059
:104230006900740079002D0046004C004F003300E7
:1042400032003A0082007000000000005400650057
:104250006D007000650072006100740075007200EE
:1042600065002D0046004C004F00330032003A003C
:104270008300A0000000000057005800300031000B
:104280001E001B0077003000300030002F0030008F
:104290003000300067003000300030007400000053
:00000001FF
